:100000000C9446000C948A000C9452000C946600E8
:100010000C948A000C948A000C948A000C948A0038
:100020000C948A000C948A000C948A000C948A0028
:100030000C948A000C948A000C948A000C948A0018
:100040000C948A000C948A000C948A000C948A0008
:100050000C948A000C948A000C948A000C948A00F8
:100060000C948A000C948A000C948A000C948A00E8
:100070000C948A000C948A000C948A000C948A00D8
:100080000C948A000C948A000C948A0011241FBEE0
:10009000CFEFD0E1DEBFCDBF0E947A000C945000BC
:0400A000F894FFCF02
:1000A4001F920F920FB60F9211248F9385B380384D
:1000B40011F485B303C085B3880F85BB8F910F906E
:0800C4000FBE0F901F9018956C
:1000CC001F920F920FB60F9211248F9385B381302C
:1000DC0011F480E885BB85B3869585BB8F910F9015
:0800EC000FBE0F901F90189544
:1000F40080EF81BB8FEF84BBEAE6F0E080818C6205
:10010400808389B7866089BF81E085BB7894FFCFFF
:040114000C94000047
:00000001FF
